:020000040800F2
:1000000010040020E1170008BD170008BF17000802
:10001000C1170008C3170008C5170008000000003A
:10002000000000000000000000000000C7170008EA
:10003000C917000800000000CB170008CD17000802
:100040000118000805180008091800080D18000814
:100050001118000815180008191800081D180008C4
:100060002118000825180008291800082D18000874
:100070003118000835180008391800083D18000824
:100080004118000800000000451800084918000841
:100090004D18000851180008551800085918000894
:1000A0005D18000861180008651800086918000844
:1000B0006D180008711800087518000879180008F4
:1000C0007D180008811800088518000889180008A4
:1000D0008D18000891180008951800089918000854
:1000E0009D180008A1180008A5180008A918000804
:1000F000AD180008B1180008B5180008000000008D
:1001000000000000B918000800000000BD18000839
:10011000C118000800000000C5180008C918000830
:10012000CD180008D1180008D5180008D918000803
:10013000DD1800080000000000000000E1180008C1
:10014000E5180008E91800080000000000000000A1
:10015000000000000000000000000000000000009F
:10016000000000000000000000000000ED18000882
:10017000F11800080000000000000000000000006E
:1001800000000000F518000800000000000000005A
:10019000000000000000000000000000000000005F
:1001A0000000000000000000F9180008FD18000819
:1001B00001190008051900080919000800000000CD
:1001C000000000000D190008000000000000000001
:1001D00011190008151900082DE9F04186B0142204
:1001E0000021684600F07BFCDFF8CC08DFF8CC5833
:1001F0000168DFF8CC78DFF8CC8841F0200101609D
:1002000041F2F034026802F0200205924BF24706F8
:100210000599026842F001020260036803F00103DD
:1002200005930599026842F004020260036803F036
:10023000040305930599026842F002020260036814
:1002400003F0020305930599026842F00802026078
:100250000022006800F00800059041F6F87105984A
:1002600000F039FC0022214600F0C4F8002231469B
:10027000384600F02FFD00220421404600F02AFD00
:1002800041F6F85100F026F800F01EF80094694697
:10029000284600F043FC00F017F8009669463846FF
:1002A00000F03CFC4FF4007100F014F804210091C0
:1002B000012200210291039101926946404600F01B
:1002C0002DFC06B0BDE8F0810120019000220292D1
:1002D0000392704700910122002102910391019243
:1002E00069464FF0904000F019BC38B500F0F1FBC2
:1002F000002203E038B500F03FF90122102100F0A0
:10030000EAFB002220214FF0904000F0E3FC0022A5
:1003100040214FF0904000F0DDFC002280214FF0A2
:10032000904000F0D7FCDFF894470022102100F045
:10033000CDFB0022202100F0C9FBDFF8845700220A
:10034000012100F057F80022022100F053F80022AA
:10035000042100F04FF800224FF4805100F04AF8D9
:1003600000224FF4005100F045F800224FF4004104
:1003700000F040F80022402100F0A8FB002280217C
:1003800000F0A4FB00224FF4807100F09FFB0022DC
:100390004FF4007100F09AFB00224FF480714FF08F
:1003A000904000F097FC00224FF400714FF0904015
:1003B00000F090FC00224FF480614FF0904000F07C
:1003C00089FC00224FF400614FF0904000F082FC65
:1003D00000224FF480514FF0904000F07BFC00224F
:1003E00000F072FBBDE8384000220421DFF8D4069B
:1003F00000F070BC284600F06DBC38B500F0BCF8C9
:1004000000F0E3F801227DE738B500F0B5F800F020
:10041000DCF800F0D4F801227AE738B500F0ACF847
:1004200000F0D3F800F0CBF800F0FAF8012275E7FD
:1004300038B500F0A1F800F0C8F800F0C0F800F0FE
:10044000EFF800F0E7F8DFF8744601226EE738B500
:1004500000F092F800F0B9F800F0B1F800F0E0F820
:1004600000F0D8F800F008F9012263E738B500F091
:1004700083F800F0AAF800F0A2F800F0D1F800F03C
:10048000C9F800F0F9F800F0F2F8DFF8345601226C
:1004900056E738B500F070F800F097F800F08FF8E4
:1004A00000F0BEF800F0B6F800F0E6F800F0DFF873
:1004B00000F011F9012247E738B500F05DF800F0CF
:1004C00084F800F07CF800F0ABF800F0A3F800F03E
:1004D000D3F800F0CCF800F0FEF800F0F7F80122B5
:1004E00036E738B500F048F800F06FF800F067F82C
:1004F00000F096F800F08EF800F0BEF800F0B7F8C3
:1005000000F0E9F800F0E2F800F011F9012223E729
:1005100038B500F031F800F058F800F050F800F06D
:100520007FF800F077F800F0A7F800F0A0F800F0EE
:10053000D2F800F0CBF800F0FAF800F0FDF8012254
:100540000FE738B500F018F800F03FF800F037F882
:1005500000F066F800F05EF800F08EF800F087F822
:1005600000F0B9F800F0B2F800F0E1F800F0E4F8BB
:1005700000F015F90122F9E6002208214FF0904021
:1005800000F0A8BB38B5FFF7F7FF00F01EF800F049
:1005900016F800F045F800F03DF800F06DF800F0B6
:1005A00066F800F098F800F091F800F0C0F800F05C
:1005B000C3F800F0F4F800F0ECF80122DBE60022CA
:1005C00020214FF0904000F085BB002210214FF019
:1005D000904000F07FBB38B5FFF7CEFFFFF7F5FF87
:1005E000FFF7EDFF00F01CF800F014F800F044F8FD
:1005F00000F03DF800F06FF800F068F800F097F8B0
:1006000000F09AF800F0CBF800F0C3F800F0FBF827
:100610000122B4E6002280214FF0904000F05ABB46
:10062000002240214FF0904000F054BB38B5FFF756
:10063000A3FFFFF7CAFFFFF7C2FFFFF7F1FFFFF7C6
:10064000E9FF00F019F800F012F800F044F800F0AB
:100650003DF800F06CF800F06FF800F0A0F800F042
:1006600098F800F0D0F800F0C9F801228BE60022DB
:100670002021204600F02EBBDFF84044002210214C
:10068000204600F027BB38B5FFF776FFFFF79DFF48
:10069000FFF795FFFFF7C4FFFFF7BCFFFFF7ECFF85
:1006A000FFF7E5FF00F017F800F010F800F03FF852
:1006B00000F042F800F073F800F06BF800F0A3F8D7
:1006C00000F09CF800F0D5F8012261E6002202213A
:1006D000284600F0FFBADFF8E8530022012128463F
:1006E00000F0F8BA38B5FFF747FFFFF76EFFFFF7E6
:1006F00066FFFFF795FFFFF78DFFFFF7BDFFFFF7E1
:10070000B6FFFFF7E8FFFFF7E1FF00F010F800F099
:1007100013F800F044F800F03CF800F074F800F032
:100720006DF800F0A6F800F09EF8012235E60022F0
:100730000421284600F0CEBA00224FF4805128460A
:1007400000F0C8BA38B5FFF717FFFFF73EFFFFF715
:1007500036FFFFF765FFFFF75DFFFFF78DFFFFF740
:1007600086FFFFF7B8FFFFF7B1FFFFF7E0FFFFF7E6
:10077000E3FF00F014F800F00CF800F044F800F08B
:100780003DF800F076F800F06EF800F0ACF80122C9
:100790000AE600224FF40041284600F09BBA0022EE
:1007A0004FF40051284600F095BA38B5FFF7E4FE43
:1007B000FFF70BFFFFF703FFFFF732FFFFF72AFFFB
:1007C000FFF75AFFFFF753FFFFF785FFFFF77EFFA5
:1007D000FFF7ADFFFFF7B0FFFFF7E1FFFFF7D9FF2E
:1007E00000F011F800F00AF800F043F800F03BF8D0
:1007F00000F079F800F070F80122DCE50022802199
:10080000204600F067BA00224021204600F062BA7C
:1008100038B5FFF7B1FEFFF7D8FEFFF7D0FEFFF7C0
:10082000FFFEFFF7F7FEFFF727FFFFF720FFFFF7B9
:1008300052FFFFF74BFFFFF77AFFFFF77DFFFFF750
:10084000AEFFFFF7A6FFFFF7DEFFFFF7D7FF00F0D1
:1008500010F800F008F800F046F800F03DF800F05D
:100860007FF80122AEE500224FF40071204600F02F
:1008700031BA00224FF48071204600F02BBA38B50F
:10088000FFF77AFEFFF7A1FEFFF799FEFFF7C8FE1C
:10089000FFF7C0FEFFF7F0FEFFF7E9FEFFF71BFFD3
:1008A000FFF714FFFFF743FFFFF746FFFFF777FF60
:1008B000FFF76FFFFFF7A7FFFFF7A0FFFFF7D9FFD5
:1008C000FFF7D1FF00F00FF800F006F800F048F84D
:1008D00000F03FF801227CE500224FF400714FF058
:1008E000904000F0F7B900224FF480714FF0904033
:1008F00000F0F0B938B5FFF73FFEFFF766FEFFF7EF
:100900005EFEFFF78DFEFFF785FEFFF7B5FEFFF7F2
:10091000AEFEFFF7E0FEFFF7D9FEFFF708FFFFF797
:100920000BFFFFF73CFFFFF734FFFFF76CFFFFF70C
:1009300065FFFFF79EFFFFF796FFFFF7D4FFFFF776
:10094000CBFF00F00DF800F004F800F044F80122AD
:1009500046E500224FF400614FF0904000F0BAB934
:1009600000224FF480614FF0904000F0B3B938B5E9
:10097000FFF702FEFFF729FEFFF721FEFFF750FE0B
:10098000FFF748FEFFF778FEFFF771FEFFF7A3FEC3
:10099000FFF79CFEFFF7CBFEFFF7CEFEFFF7FFFE53
:1009A000FFF7F7FEFFF72FFFFFF728FFFFF761FFC5
:1009B000FFF759FFFFF797FFFFF78EFFFFF7D0FF15
:1009C000FFF7C7FF00F007F8002200F07DF8BDE850
:1009D0003840012209E500224FF480514FF0904049
:1009E00000F078B938B500F074F80122102100F059
:1009F00072F80122202100F06EF80122402100F05F
:100A00006AF80122802100F066F82C4C01221021A6
:100A100000F05CF80122202100F058F8284D012256
:100A20000121FFF7E7FC01220221FFF7E3FC01228D
:100A30000421FFF7DFFC01224FF48051FFF7DAFCBD
:100A400001224FF40051FFF7D5FC01224FF4004181
:100A5000FFF7D0FC0122402100F038F8012280216C
:100A600000F034F801224FF4807100F02FF80122D9
:100A70004FF4007100F02AF801224FF4807100F069
:100A80002AF801224FF4007100F025F801224FF4FA
:100A9000806100F020F801224FF4006100F01BF8A3
:100AA00001224FF4805100F016F8012200F00CF8FA
:100AB000BDE83840012298E44C100240000800488C
:100AC00000040048000C00484FF48051204600F01C
:100AD00001B9012208214FF0904000F0FBB810B599
:100AE000044610460A460146204600F009F9204611
:100AF00010BD0EE002684368024408305FEAC37C20
:100B000044BF4B445B1E52F804CB43F804CB091F8F
:100B1000F9D150F8041B0029ECD170472DE9F84FAA
:100B200000276F4A6F4B4FF00F0805460E4636E020
:100B30006D4CA54214BF062405248C406B4944EA41
:100B40000E0441F82C40C143D2F808C0746801EA91
:100B50000C0CE40248BF40EA0C0CC2F808C0D2F802
:100B60000CC0746801EA0C0CA40248BF40EA0C0CEB
:100B7000C2F80CC0D2F804C0746801EA0C0CA403DB
:100B800048BF40EA0C0CC2F804C0D2F800C0746838
:100B900001EA0C01E40348BF014311607F1C316886
:100BA00031FA07F000F094800124BC4014EA0100FF
:100BB000F4D04FEA470C032101FA0CF16FEA010E61
:100BC000716801F00309B9F1010F1CBF01F00301C5
:100BD000022912D1A968D6F80C900EEA010109FA8F
:100BE0000CF949EA0101A960696821EA0404716805
:100BF000C1F30011B9400C436C60B900347904F0C2
:100C00000304032C21D0EC68D6F808900EEA040403
:100C100009FA0CF949EA0404EC60347904F003049D
:100C2000022C12D1FC0805EB840401F01C09D4F855
:100C300020A008FA09FB2AEA0B0AD6F810B00BFA32
:100C400009F949EA0A09C4F820902C680EEA040E52
:100C5000347904F0030404FA0CF444EA0E0CC5F8E9
:100C600000C0746814F4403F98D0D3F800C01F4C03
:100C70004CF0010CC3F800C04FEA970CD3F800E029
:100C80000EF0010ECDF800E001F00C01DDF800E0FF
:100C900054F82CE008FA01F42EEA040EB5F1904F56
:100CA00008BF002413D0124CA54208BF01240ED067
:100CB000104CA54208BF022409D00F4CA54208BF22
:100CC000032404D00D4CA5427FF432AF042434E752
:100CD000BDE8F18F0AB18161704781627047000001
:100CE0000004014060100240001400480800014068
:100CF0000004004800080048000C004800100048AC
:100D000062F30F2262F31F42401810F0030308D071
:100D1000C91A1FD3DB0748BF00F8012D28BF20F8F0
:100D2000022D130030B414461546103928BF20E9AF
:100D30003C00FAD8490728BF20E90C0048BF40F81A
:100D4000042D890028BF20F8022D48BF00F8012D8E
:100D500030BC7047C91818BF00F8012DCB0728BF59
:100D600000F8012D704700002DE9F84304006DD014
:100D70002078DFF8B865C10717D500F0CDF90CD1A0
:100D800001F0030103290AD06068B0F5803F2AD141
:100D9000306840F48030306037E00828F4D13068A3
:100DA000810302D56068002850D02178880759D582
:100DB00000F0B2F943D101F00301022941D0E0680B
:100DC00000286AD0316841F48071316000F0C8FABF
:100DD0000546306841055DD400F0C2FA401B032887
:100DE000F7D303205FE1B0F5A02F306806D140F4BF
:100DF00080203060316841F4803105E020F480309B
:100E00003060316821F480213160606858B100F0B1
:100E1000A7FA054630688103C7D400F0A1FA401B49
:100E20006528F7D3DDE700F09BFA054630688103BB
:100E3000BBD500F095FA401B6528F7D3D1E704280D
:100E4000BDD13068410503D5E068002800F05A8123
:100E500000F05AF9DFF8E004006800F087FA002893
:100E600040F050812078DFF8D474010734D56069F0
:100E70000028786821D040F00100786000F070FA16
:100E800005467868810727D400F06AFA401B0328DA
:100E9000F7D3A6E700F038F9E4E7306820F4807073
:100EA000306000F05DFA054630684105DAD500F0A3
:100EB00057FA401B0328F7D393E7400840007860B7
:100EC00000F04EFA05467868810705D500F048FA2B
:100ED000401B0328F7D384E72078410763D5B06D22
:100EE0000025C10009D4B06D40F08050B0650125E7
:100EF000B06D00F0805000900098DFF84484D8F87E
:100F00000000C10513D4D8F8000040F48070C8F880
:100F1000000000F025FA8146D8F80000C10506D48B
:100F200000F01EFAA0EB09000328F5D359E7A068EA
:100F3000012804D1386840F00100386010E005282D
:100F4000386806D140F004003860396841F001018A
:100F500005E0400840003860396821F0040139603C
:100F6000A06841F2893860B100F0FAF9814638682A
:100F7000810713D400F0F4F9A0EB09004045F6D343
:100F80002FE700F0EDF981463868810706D500F0BB
:100F9000E7F9A0EB09004045F6D322E71DB1B06D9B
:100FA00020F08050B0652078810621D5A069002806
:100FB000B8680ED040F00100B86000F0D1F90546E5
:100FC000B868810714D400F0CBF9401B0328F7D38D
:100FD00007E740084000B86000F0C2F90546B8686D
:100FE000810705D500F0BCF9401B0328F7D3F8E6CC
:100FF000E069002856D0B16801F00C010C2954D0EA
:101000000228306820F0807030603AD100F0A8F9F2
:1010100005463068810105D500F0A2F9401B032880
:10102000F7D3DEE6F068DFF81C13226A0840616A35
:101030001043491E40EA0110226BA16A520840EA9F
:101040000120616B521E490840EA4250491E40EAA5
:101050004160E16A40EAC160F060306840F0807051
:101060003060F16841F08071F16000F079F9044678
:101070003068810116D400F073F9001B0328F7D300
:10108000AFE600F06DF904463068810105D500F047
:1010900067F9001B0328F7D3A3E6F068DFF8A8126E
:1010A0000840F0600020BDE8F28301282AD0F068F3
:1010B000226A00F00301914201BF00F0F0011031FB
:1010C000626AB1EB021F1DD1A26A00F4FE41B1EBCE
:1010D000022F02BF00F07841E26AB1EBC26F11D17A
:1010E000226B00F4C00101F500115208B1EB425F20
:1010F00008D1616B00F0C06000F100704908B0EBEE
:10110000416FCFD00120CEE77068216920F0FE400A
:1011100040EA016070607047B068F16800F00C0050
:101120000C2870472DE9F84F04460026002C6CD09F
:10113000DFF818723868894600F00F00484506D27B
:1011400000F0BFF8386800F00F0048455DD1206816
:10115000DFF8D851C10741F2893858D56168DFF806
:10116000F0B103294FF0080A27D129688A014CD52C
:10117000EA68E968C1F30311491C02F00302032A7B
:101180000CBFDFF8D021DFF8AC21B2FBF1F2E96847
:10119000C1F306215143EA68C2F34162521C520076
:1011A000B1FBF2F1594516D3AA6812F0F00F0DD039
:1011B000810710D5A06870B908E00229286822D1FB
:1011C000810322D500F083F8584504D3A8686AF358
:1011D0000710A8608026A9686068890840EA810134
:1011E000A96000F0BDF88246A868616800F00C00B4
:1011F000B0EB810F0BD000F0B3F8A0EB0A00404534
:10120000F2D303205BE04105DCD4012057E02068E5
:10121000810714D5400703D5A96841F4E061A960AE
:101220002078010704D5A968072060F30D21A96083
:10123000A968A06821F0F0010143A96005E0802EB3
:1012400003D1A86820F0F000A860386800F00F0013
:1012500081450FD200F035F800F082F80646386874
:1012600000F00F00484505D000F07AF8801B40459B
:10127000F5D3C6E72078410705D5AA68E06822F4CF
:10128000E0620243AA602178080706D5A9682069B0
:1012900021F4605141EAC001A96000F018F8AA6881
:1012A0002D49C2F30312895C214A01F01F01C84095
:1012B0001060BDE8F24F2048006800F057B8BDE864
:1012C000F28F3968090949EA0111396070472348EA
:1012D000016801F00C01042901D11648704701682A
:1012E00001F00C01082901D11A487047016801F08A
:1012F0000C010C2918D142684168C1F30311491C43
:1013000002F00302032A0CBF124A0A4AB2FBF1F2AE
:1013100041684068C0F34160C1F30621401C51435D
:101320004000B1FBF0F07047002070470010024011
:101330000C0000200024F400040000209010024063
:10134000007000400C809F01FCFFEEFE0020024078
:1013500001B4C40400127A004817000808100240C3
:1013600001480068704700BF0000002070B50E4EB5
:101370000446B0680025A0B14FF47A710B4AB1FB66
:10138000F0F11068B0FBF1F000F04AF848B9102C09
:1013900007D2002221464FF0FF3000F023F874609E
:1013A00000E00125284670BD000000200C00002050
:1013B0000901020002D4234881547047224B02F0F5
:1013C0000F021A4402F8041C7047204B19684FF6AC
:1013D000FF020002114000F4E06008431C4908438A
:1013E0001860704770B5194B1C68C4F302230124C0
:1013F000C3F10705052D2EBF0F2504FA05F56D1E57
:101400001E1D072E34BF0023DB1E2940994004FA1D
:1014100003F3BDE870405B1E1A401143C8E70000AB
:10142000401EB0F1807F01D30120704709490A4A6C
:1014300048600023F02010708B60072008600020B7
:101440007047000000E400E018ED00E00CED00E063
:101450000000FA0510E000E023ED00E080B500F0A8
:10146000A7F800F06DF8FEF7B7FEFFF7BBFA4FF4F0
:101470007A7000F0ADF8FEF738FF00F05DF8FEF787
:1014800039FF00F059F8FEF7B8FF00F055F8FEF705
:10149000BBFF00F051F8FEF7C0FF00F04DF8FEF77B
:1014A000C7FF00F049F8FEF7D2FF00F045F8FEF75D
:1014B000DDFF00F041F8FEF7ECFF00F03DF8FEF72D
:1014C000FBFF00F039F8FFF70CF800F035F8FFF7F4
:1014D0001FF800F031F8FFF734F800F02DF8FFF7AF
:1014E00051F800F029F8FFF776F800F025F8FFF73B
:1014F0009DF800F021F8FFF7C6F800F01DF8FFF79F
:10150000F1F800F019F8FFF71DF900F015F8FFF7F2
:101510004CF900F011F8FFF77BF900F00DF8FFF738
:10152000AEF900F009F8FFF7E5F900F005F8FFF76C
:101530001EFA00F001F898E74FF4967000F048B8F2
:1015400000B593B03822002105A8FFF7C8FA14228D
:1015500000216846FFF7C3FA002000F04DF84FF471
:1015600080310691012003210D9105900222552121
:101570000C920E920F9110921192129205A8FFF701
:10158000F3FB08B100F011F80F2003210090019146
:10159000002202920392049204216846FFF7C2FDE2
:1015A00008B100F002F813B000BD72B6FEE700000B
:1015B000032010B5FFF709FF0F20FFF7D7FE002427
:1015C000002814BF012400F06DF8204610BD000073
:1015D00038B50446FFF7C4FE14F1010F054602D0EA
:1015E000044988680419FFF7BBFE401BA042FAD3E8
:1015F00031BD00BF0000002030B53222DFF8983046
:10160000DFF89050DFF88810012448B900F01DF889
:1016100020F48070286016D100F01EF80CD412E07F
:10162000B0F5007F0AD100F010F840F48070286017
:1016300009D100F011F806D5032030BD0A68022058
:1016400060F34A220A60002030BD086800F4C060E0
:10165000B0F5806F28687047086864F34A20086016
:101660001B68DFF838405A43B2FBF4F0401C00E03E
:10167000401E4A69530501D50028F9D14869410542
:1016800070470748016841F48041016070470000DD
:1016900000700040807000400C00002040420F00AD
:1016A000087000400B4882B0816841F00101816000
:1016B000816801F0010100910099026842F08052B6
:1016C0000260006800F080500090009802B0FFF7C0
:1016D000D8BF00BF5810024010B5074979441831EF
:1016E000064C7C44163404E00A68081D11448847FF
:1016F0000146A142F8D110BD2C0000003C000000C2
:101700004EF68851CEF20001086840F4700008607F
:10171000BFF34F8FBFF36F8F4FF00170E1EE100AF0
:1017200070470000CFF3FFFF10000000C40000006E
:1017300000000020000000000248016841F4700130
:101740000160704788ED00E000000000000000002C
:10175000010203040607080900F00DF8002801D073
:10176000FFF7BAFFAFF300800020AFF30080FFF770
:1017700075FE00F002F80120704700F001B800008B
:101780000746384600F002F8FBE7000080B5AFF3EB
:101790000080024A11001820ABBEFBE726000200C1
:1017A0000548014603B4684680F30988AFF300801A
:1017B000FFF7A6FFFFF7D0FFA5EDF5FEFEE7FEE77A
:1017C000FEE7FEE7FEE770477047704700F000B89D
:1017D00002490A68886882180A6070470000002081
:1017E000014880470148004739170008A117000841
:1017F0000000000010000000010000000024F400C0
:10180000FFF7FEBFFFF7FEBFFFF7FEBFFFF7FEBF0C
:10181000FFF7FEBFFFF7FEBFFFF7FEBFFFF7FEBFFC
:10182000FFF7FEBFFFF7FEBFFFF7FEBFFFF7FEBFEC
:10183000FFF7FEBFFFF7FEBFFFF7FEBFFFF7FEBFDC
:10184000FFF7FEBFFFF7FEBFFFF7FEBFFFF7FEBFCC
:10185000FFF7FEBFFFF7FEBFFFF7FEBFFFF7FEBFBC
:10186000FFF7FEBFFFF7FEBFFFF7FEBFFFF7FEBFAC
:10187000FFF7FEBFFFF7FEBFFFF7FEBFFFF7FEBF9C
:10188000FFF7FEBFFFF7FEBFFFF7FEBFFFF7FEBF8C
:10189000FFF7FEBFFFF7FEBFFFF7FEBFFFF7FEBF7C
:1018A000FFF7FEBFFFF7FEBFFFF7FEBFFFF7FEBF6C
:1018B000FFF7FEBFFFF7FEBFFFF7FEBFFFF7FEBF5C
:1018C000FFF7FEBFFFF7FEBFFFF7FEBFFFF7FEBF4C
:1018D000FFF7FEBFFFF7FEBFFFF7FEBFFFF7FEBF3C
:1018E000FFF7FEBFFFF7FEBFFFF7FEBFFFF7FEBF2C
:1018F000FFF7FEBFFFF7FEBFFFF7FEBFFFF7FEBF1C
:10190000FFF7FEBFFFF7FEBFFFF7FEBFFFF7FEBF0B
:08191000FFF7FEBFFFF7FEBF69
:04000005080017A137
:00000001FF
